:101C000012C02BC02AC029C028C027C026C025C0AA
:101C100024C023C022C021C020C01FC01EC01DC0C0
:101C20001CC01BC01AC011241FBECFE5D4E0DEBF0C
:101C3000CDBF10E0A0E6B0E0E6EFFFE102C0059006
:101C40000D92A236B107D9F711E0A2E6B0E001C0CB
:101C50001D92AA36B107E1F74BC0D2CFEF92FF92A7
:101C60000F931F93EE24FF2487015F9915C00894FA
:101C7000E11CF11C011D111D81E0E81682E1F8064E
:101C80008AE7080780E0180728F0E0916200F091E9
:101C9000630009955F9BEBCF8CB1992787FD9095E9
:101CA0001F910F91FF90EF9008955D9BFECF8CB92F
:101CB0000895D4DF803221F484E1F7DF80E1F5DF9D
:101CC00008950895CF93C82FC9DF803231F484E19D
:101CD000ECDF8C2FEADF80E1E8DFCF910895CF932E
:101CE000882321F0C82FBADFC150E9F7CF910895BA
:101CF000CFE5D4E0DEBFCDBF000010BC83E389B9DF
:101D000088E18AB986E880BDBD9A1092680130E208
:101D10002FE088B3832788BB80E090E00197F1F73C
:101D2000215027FFF6CF20E12093680197DF803311
:101D300009F444C08133A1F491DFC82F8032B1F798
:101D400084E1B3DF81E4B1DF86E5AFDF82E5ADDFBB
:101D50008C2FABDF89E4A9DF83E5A7DF80E52EC107
:101D6000803429F47BDF863848F178DF27C081345E
:101D700071F474DF803811F482E028C1813811F4E5
:101D800081E024C1823809F020C182E11FC1823480
:101D900011F484E103C0853419F485E0A0DF0EC09E
:101DA000803561F0813551F0823541F0853541F45F
:101DB00055DF8093640052DF809365007ADFB6CFF1
:101DC000863519F484E08BDF00C1843609F09DC0AC
:101DD00045DF8093670142DF80936601809169014E
:101DE0008E7F809369013ADF853429F480916901FF
:101DF000816080936901C0E0D0E08091660190919C
:101E00006701C817D90770F406E610E027DFF8016C
:101E100081938F0121968091660190916701C81787
:101E2000D907A0F31BDF803209F080CF80916901D0
:101E300080FF26C0C0E0D0E08091660190916701EC
:101E4000C817D90708F05FC006E610E0F8016191F5
:101E50008F018091640090916500C2D080916400F0
:101E6000909165000196909365008093640021969F
:101E70008091660190916701C817D90738F343C074
:101E8000F894E199FECF1127E0916400F09165008C
:101E9000EE0FFF1FC6E6D0E08091660190916701CA
:101EA00080FF01C00196103051F422D003E000936E
:101EB0005700E8951DD001E100935700E89509907F
:101EC000199016D001E000935700E8951395103251
:101ED00058F011270DD005E000935700E89508D081
:101EE00001E100935700E8953296029739F0DBCF75
:101EF0000091570001700130D9F30895103011F0AE
:101F00000296E7CF112484E159C0843709F049C013
:101F1000A5DE80936701A2DE809366019FDE90912B
:101F20006901853421F49160909369010DC09E7F11
:101F3000909369018091640090916500880F991FCA
:101F4000909365008093640089DE803209F0EECEC4
:101F500084E1ABDEC0E0D0E0809166019091670142
:101F6000C817D90760F58091690180FF06C080918C
:101F70006400909165002CD008C0869580FD06C055
:101F8000E0916400F091650084918FDE809164009F
:101F9000909165000196909365008093640021966E
:101FA000DBCF853779F45ADE803209F0BFCE84E189
:101FB0007CDE8EE17ADE83E978DE87E076DE80E122
:101FC00074DEB4CE863709F0B1CE80E07BDEAECED3
:101FD000E199FECF9FBB8EBBE09A99278DB3089500
:101FE000E199FECF9FBB8EBB6DBB0FB6F894E29A12
:061FF000E19A0FBE089506
:021FF600800069
:0400000300001C00DD
:00000001FF
